:020000023000CC
:10E000000D94F6F20D941FF30D941FF30D941FF36E
:10E010000D941FF30D941FF30D941FF30D941FF334
:10E020000D941FF30D941FF30D941FF30D941FF324
:10E030000D941FF30D941FF30D941FF30D941FF314
:10E040000D941FF30D941FF30D941FF30D941FF304
:10E050000D941FF30D941FF30D941FF30D941FF3F4
:10E060000D941FF30D941FF30D941FF30D941FF3E4
:10E070000D941FF30D941FF30D941FF30D941FF3D4
:10E080000D941FF30D941FF30D941FF30D941FF3C4
:10E090000D941FF30D941FF30D941FF30D941FF3B4
:10E0A0000D941FF30D941FF30D941FF30D941FF3A4
:10E0B0000D941FF30D941FF30D941FF30D941FF394
:10E0C0000D941FF30D941FF30D941FF30D941FF384
:10E0D0000D941FF30D941FF30D941FF30D941FF374
:10E0E0000D941FF341546D65676132353630004140
:10E0F000726475696E6F206578706C6F72657220DE
:10E1000073746B3530305632206279204D4C530099
:10E11000426F6F746C6F616465723E004875683F52
:10E1200000436F6D70696C6564206F6E20203D2028
:10E1300000435055205479706520202020203D2038
:10E14000005F5F4156525F415243485F5F203D2070
:10E1500000415652204C69624320566572203D2092
:10E16000004743432056657273696F6E20203D203F
:10E1700000435055207369676E61747572653D2068
:10E18000004C6F77206675736520202020203D208D
:10E1900000486967682066757365202020203D204F
:10E1A00000457874206675736520202020203D206E
:10E1B000004C6F636B2066757365202020203D2026
:10E1C00000417072203133203230313200312E362E
:10E1D0002E3700342E332E33005623202020414486
:10E1E00044522020206F7020636F6465202020201F
:10E1F00020696E737472756374696F6E20616464F4
:10E2000072202020496E74657272757074006E6F92
:10E2100020766563746F7200726A6D702020006AE8
:10E220006D7020005768617420706F72743A0050EE
:10E230006F7274206E6F7420737570706F72746576
:10E2400064004D7573742062652061206C65747480
:10E2500065720020005772697474696E67204545C5
:10E260000052656164696E6720454500656570729E
:10E270006F6D206572726F7220636F756E743D00F2
:10E28000504F525400303D5A65726F206164647281
:10E290006573732063747273003F3D435055207360
:10E2A0007461747300403D454550524F4D20746574
:10E2B000737400423D426C696E6B204C45440045CE
:10E2C0003D44756D7020454550524F4D00463D44CC
:10E2D000756D7020464C41534800483D48656C7050
:10E2E000004C3D4C69737420492F4F20506F72745D
:10E2F0007300513D517569742026206A756D702038
:10E30000746F20757365722070676D00523D44759F
:10E310006D702052414D00563D73686F7720696ED5
:10E320007465727275707420566563746F727300D1
:10E33000593D506F727420626C696E6B002A0052F6
:10E340004553455400494E543000494E543100491C
:10E350004E543200494E543300494E543400494E15
:10E36000543500494E543600494E54370050434905
:10E370004E5430005043494E5431005043494E549E
:10E3800032005744540054494D45523020434F4DBC
:10E3900050410054494D45523020434F4D504200AA
:10E3A00054494D455230204F56460054494D455230
:10E3B0003120434150540054494D45523120434F80
:10E3C0004D50410054494D45523120434F4D50422C
:10E3D0000054494D45523120434F4D50430054495C
:10E3E0004D455231204F56460054494D455232203A
:10E3F000434F4D50410054494D45523220434F4DFB
:10E4000050420054494D455232204F56460054491F
:10E410004D45523320434150540054494D455233E9
:10E4200020434F4D50410054494D45523320434FF6
:10E430004D50420054494D45523320434F4D5043B7
:10E440000054494D455233204F56460054494D45DE
:10E45000523420434150540054494D4552342043D6
:10E460004F4D50410054494D45523420434F4D507B
:10E47000420054494D45523420434F4D50430054BF
:10E48000494D455234204F56460054494D4552356A
:10E4900020434150540054494D45523520434F4D7F
:10E4A00050410054494D45523520434F4D50420094
:10E4B00054494D45523520434F4D50430054494D2A
:10E4C000455235204F564600555341525430205244
:10E4D000580055534152543020554452450055532D
:10E4E0004152543020545800555341525431205217
:10E4F000580055534152543120554452450055530C
:10E5000041525431205458005553415254322052F4
:10E5100058005553415254322055445245005553EA
:10E5200041525432205458005553415254332052D2
:10E5300058005553415254332055445245005553C9
:10E5400041525433205458005350492053544300EF
:10E5500041444300414E414C4F4720434F4D5000F2
:10E560004545205245414459005457490053504DA8
:10E57000205245414459002A003FE345E34AE34F16
:10E58000E354E359E35EE363E368E36DE374E37B41
:10E59000E382E3E9E3F6E303E4ABE3B7E3C4E3D107
:10E5A000E3DEE386E393E3A0E348E5C8E4D2E4DEF8
:10E5B000E454E550E560E50EE41AE427E434E44170
:10E5C000E4E8E4F2E4FEE469E56DE54CE458E46572
:10E5D000E472E47FE48AE496E4A3E4B0E4BDE408F2
:10E5E000E512E51EE528E532E53EE50011241FBEF3
:10E5F000CFEFD1E2DEBFCDBF01E00CBF12E0A0E063
:10E60000B2E0EEE8FFEF03E00BBF02C007900D920F
:10E61000A030B107D9F712E0A0E0B2E001C01D922E
:10E62000AC30B107E1F70F94FBF40D94C5FF01E2A4
:10E630000EBF0FEF0DBF11241FBE0D94FBF40D9400
:10E6400000F020E030E040ED57E005C0FA013197DE
:10E65000F1F72F5F3F4F28173907C0F308959C014A
:10E66000442737FD4095542FDA01C901860F911DCB
:10E67000A11DB11DABBFFC018791882369F0809378
:10E68000C6008091C00086FFFCCF8091C0008064EE
:10E690008093C0006F5FE8CF08958DE08093C6003F
:10E6A0008091C00086FFFCCF8091C0008064809381
:10E6B000C0008AE08093C6008091C00086FFFCCF36
:10E6C0008091C00080648093C00008950F942FF360
:10E6D0000F944DF30895FC019081992359F0909384
:10E6E000C6008091C00086FFFCCF8091C00080648E
:10E6F0008093C0003196992379F70895282F982F99
:10E7000092959F70892F805D8A3308F0895F80938E
:10E71000C6008091C00086FFFCCF8091C00080645D
:10E720008093C000822F8F70982F905D9A3308F0ED
:10E73000995F9093C6008091C00086FFFCCF8091C6
:10E74000C00080648093C00008959C01FB01853661
:10E7500091051CF46330710594F0C90164E670E022
:10E760000F9466FF605D7F4F6093C6008091C0008C
:10E7700086FFFCCF8091C00080648093C0002B3066
:10E78000310514F43297B4F0C90164E670E00F94D7
:10E7900066FF6AE070E00F9466FF605D7F4F6093F4
:10E7A000C6008091C00086FFFCCF8091C0008064CD
:10E7B0008093C000C9016AE070E00F9466FFC096C4
:10E7C0008093C6008091C00086FFFCCF8091C0007E
:10E7D00080648093C0000895282F277020642093C0
:10E7E0007C0020917B0086958695869590E08170CF
:10E7F000907033E0880F991F3A95E1F7277F282B17
:10E8000020937B0080917A00806480937A008091CD
:10E810007A0086FDFCCF2091780040917900942FFA
:10E8200080E030E0282B392BC90108951F93182F61
:10E8300080E892EE60E00F942FF31093C600809171
:10E84000C00086FFFCCF8091C00080648093C00030
:10E850000F944DF31F9108952F923F924F925F9224
:10E860006F927F928F929F92AF92BF92CF92DF92E0
:10E87000EF92FF920F931F93DF93CF93CDB7DEB745
:10E8800062970FB6F894DEBF0FBECDBF382E622E52
:10E89000CA01DB015C016D01772460E2262E2E01A6
:10E8A0000894411C511C8BC081E0A81680E0B8067A
:10E8B00081E0C80680E0D80628F0C601AA27BB2759
:10E8C0000F947EF3BB27AD2D9C2D8B2D0F947EF3E3
:10E8D0008A2D0F947EF32092C6008091C00086FF9F
:10E8E000FCCF8091C00080648093C0009DE2909333
:10E8F000C6008091C00086FFFCCF8091C00080647C
:10E900008093C0002092C6008091C00086FFFCCF9B
:10E910008091C00080648093C000198286017501D7
:10E9200088249924A1E03A1651F03A1620F0B2E07A
:10E930003B1661F409C00BBFF701779007C0C70110
:10E940000F94AFFF782E02C0F7017080872D0F94CF
:10E950007EF32092C6008091C00086FFFCCF80919C
:10E96000C00080648093C000872D8052F401EF7056
:10E97000F0708F3520F4E40DF51D708204C0E40DB5
:10E98000F51D8EE280830894E11CF11C011D111D10
:10E990000894811C911C90E18916910409F0C2CF62
:10E9A00080E190E0A0E0B0E0A80EB91ECA1EDB1E18
:10E9B000198AC2010F946BF30F944DF36A94662089
:10E9C00009F072CF62960FB6F894DEBF0FBECDBFCE
:10E9D000CF91DF911F910F91FF90EF90DF90CF903B
:10E9E000BF90AF909F908F907F906F905F904F906F
:10E9F0003F902F9008952F923F924F925F926F9287
:10EA00007F928F929F92AF92BF92CF92DF92EF92BE
:10EA1000FF920F931F93DF93CF93CDB7DEB7C95308
:10EA2000D1400FB6F894DEBF0FBECDBF279A2F9A04
:10EA30008091C00082608093C00080E18093C40018
:10EA400088E18093C1000000EE24FF248701B4E038
:10EA5000AB2EB12CCC24DD2424C0C5010197F1F7E5
:10EA60000894E11CF11C011D111D21E2E2162EE4A7
:10EA7000F20620E0020720E0120718F0A1E0CA2EFB
:10EA8000D12CC801B70128E53BE140E050E00F94EC
:10EA900079FF611571058105910519F485B18058DB
:10EAA00085B98091C00087FD03C0C114D104A9F2CB
:10EAB000A6014F5F5F4FC25EDE4F59834883CE5140
:10EAC000D140C25EDE4F88819981CE51D1400197FD
:10EAD00011F00D9448FFC05DDE4F19821882C053BB
:10EAE000D14060E0C15DDE4F1882CF52D140AA24F0
:10EAF000BB24C05EDE4F188219821A821B82C0526C
:10EB0000D140EE24FF2487010BBFF7010791169136
:10EB1000C85CDE4F19830883C853D1400D9443FF6E
:10EB2000C25EDE4F28813981CE51D140213031057E
:10EB300009F52091C600C25EDE4F19821882CE51BF
:10EB4000D14022C02F5F3F4F4F4F5F4F213082E1B6
:10EB500038078AE7480780E0580780F0C85CDE4F36
:10EB6000E881F981C853D140EF5FFF4F19F0EE27DC
:10EB7000FF27099420E030E040E050E08091C000A1
:10EB800087FFE0CF2091C600213209F094C6089497
:10EB9000A11CB11C13E0A116B10409F08EC600E05F
:10EBA00010E018C041E24093C6008091C00086FF8B
:10EBB000FCCF8091C00080648093C0002F5F3F4FE6
:10EBC0002931310579F70F944DF30F5F1F4F053051
:10EBD000110519F020E030E0E5CF10920802109204
:10EBE000090210920A0210920B0210920402109273
:10EBF0000502109206021092070210920002109273
:10EC0000010210920202109203028FEE90EE60E079
:10EC10000F9466F380E191EE60E00F942FF3809102
:10EC2000C00087FFFCCF9091C600903608F09F751A
:10EC30009032B8F09093C6008091C00086FFFCCF60
:10EC40008091C00080648093C00080E28093C60001
:10EC50008091C00086FFFCCF8091C00080648093CB
:10EC6000C000983409F4DBC19934B8F4923409F443
:10EC70005DC1933458F4903319F1903308F418C6F9
:10EC80009F33A1F1903409F013C6BDC0953409F447
:10EC900074C1963409F00CC69CC1923509F42FC298
:10ECA000933538F49C3409F4F9C1913509F000C664
:10ECB0001CC2963509F449C2993509F0F9C59CC4BE
:10ECC00085E892EE62E00F9466F3109204021092CF
:10ECD000050210920602109207021092080210928A
:10ECE000090210920A0210920B0217C189E992EEF2
:10ECF00062E00F9466F38FEE90EE60E00F9466F39F
:10ED000081E291EE60E00F942FF381EC91EE60E0F0
:10ED10000F9466F381E391EE60E00F942FF384EE9D
:10ED200090EE60E00F9466F381E491EE60E00F9462
:10ED30002FF386E090E061E070E00F94A5F30F946C
:10ED40004DF381E691EE60E00F942FF383ED91EEA9
:10ED500060E00F9466F381E591EE60E00F942FF38D
:10ED60008DEC91EE60E00F9466F381E791EE60E048
:10ED70000F942FF38EE10F947EF388E90F947EF3C6
:10ED800081E00F947EF30F944DF381E891EE60E003
:10ED90000F942FF319E0E0E0F0E010935700E491B6
:10EDA0008E2F0F947EF30F944DF381E991EE60E086
:10EDB0000F942FF3E3E0F0E010935700E4918E2FCF
:10EDC0000F947EF30F944DF381EA91EE60E00F947F
:10EDD0002FF3E2E0F0E010935700E4918E2F0F94B0
:10EDE0007EF30F944DF381EB91EE60E00F942FF3DF
:10EDF000E1E0F0E0109357001491812F0F947EF31F
:10EE00000F944DF307CF85EA92EE62E00F9466F31C
:10EE100085E592EE60E00F9466F30F944DF300E009
:10EE200010E019C0C8016F2D0F94B7FFFF2031F417
:10EE300083E592EE60E00F942FF30BC0F092C600D2
:10EE40008091C00086FFFCCF8091C00080648093D9
:10EE5000C0000F5F1F4FC80181519F41AA2797FD36
:10EE6000A095BA2FABBFFC01F7905AE2F51621F03E
:10EE700082E000301807B1F60F944DF30F944DF374
:10EE800081E692EE60E00F9466F30F944DF3CC248C
:10EE9000DD2400E010E01EC0C8010F94AFFFF82E83
:10EEA000882331F483E592EE60E00F942FF30BC0DA
:10EEB0008093C6008091C00086FFFCCF8091C00087
:10EEC00080648093C000FE1419F00894C11CD11C0A
:10EED0000F5F1F4FC80181519F41AA2797FDA09541
:10EEE000BA2FABBFFC01E7909AE2E91621F0A2E04D
:10EEF00000301A0789F60F944DF30F944DF38CE60A
:10EF000092EE60E00F942FF3C60161E070E00F9481
:10EF1000A5F30F944DF30F944DF31092000210924D
:10EF20000102109202021092030274CE83EB92EE61
:10EF300062E00F9466F3279A2F9A16C02F9880E00C
:10EF400090E0E0EDF7E03197F1F701968436910516
:10EF5000C1F72F9A80E090E0E0EDF7E03197F1F70C
:10EF6000019684369105C1F78091C00087FFE6CFF6
:10EF70008091C00087FFFCCF95C48FEB92EE62E0DA
:10EF80000F9466F3409100025091010260910202D9
:10EF90007091030281E020E10F942CF48091000233
:10EFA00090910102A0910202B091030280509F4F04
:10EFB000AF4FBF4F8093000290930102A0930202D3
:10EFC000B093030280509041A040B04008F422CE9C
:10EFD000A4CF8DEC92EE62E00F9466F340910402B0
:10EFE00050910502609106027091070280E020E1D5
:10EFF0000F942CF48091040290910502A0910602D6
:10F00000B091070280509F4FAF4FBF4F80930402D3
:10F0100090930502A0930602B0930702FBCD8AED00
:10F0200092EE62E00F9466F385E892EE60E00F9452
:10F0300066F389E992EE60E00F9466F385EA92EE5A
:10F0400060E00F9466F383EB92EE60E00F9466F35A
:10F050008FEB92EE60E00F9466F38DEC92EE60E041
:10F060000F9466F38AED92EE60E00F9466F381EE02
:10F0700092EE60E00F9466F382EF92EE60E00F9400
:10F0800066F38CE093EE60E00F9466F387E193EE15
:10F0900060E00F9466F380E393EEB9CD81EE92EEDB
:10F0A00062E00F9466F381E40F9416F482E40F9407
:10F0B00016F483E40F9416F484E40F9416F485E4B4
:10F0C0000F9416F486E40F9416F487E40F9416F464
:10F0D00088E40F9416F48AE40F9416F48BE40F94EA
:10F0E00016F48CE40F9416F495CD82EF92EE62E064
:10F0F0000F9466F399249394AA24BB2445C48CE00E
:10F1000093EE62E00F9466F3409108025091090279
:10F1100060910A0270910B0282E020E10F942CF4BE
:10F120008091080290910902A0910A02B0910B020D
:10F1300080509F4FAF4FBF4F8093080290930902BA
:10F14000A0930A02B0930B0265CD87E193EE62E0D3
:10F150000F9466F384EE90EE60E00F9466F389ED11
:10F1600091EE60E00F9466F309E715EECC5DDE4F9B
:10F1700019830883C452D140662477244301CA5DB1
:10F18000DE4F19821882C652D140A40193015695D0
:10F19000479537952795C85DDE4F288339834A8385
:10F1A0005B83C852D140CA5DDE4F48815981C65247
:10F1B000D1404F5F5F4FCA5DDE4F59834883C652CF
:10F1C000D140CA0162E070E00F94A5F350E2509381
:10F1D000C6008091C00086FFFCCF8091C000806493
:10F1E0008093C0008DE28093C6008091C00086FFAE
:10F1F000FCCF8091C00080648093C00090E2909327
:10F20000C6008091C00086FFFCCF8091C000806462
:10F210008093C000C85DDE4FE880F9800A811B81C1
:10F22000C852D140BB27A12F902F8F2D0F947EF372
:10F23000C85DDE4F8881C852D1400F947EF370E2E2
:10F24000F72EF092C6008091C00086FFFCCF80911F
:10F25000C00080648093C0000DE30093C6008091DD
:10F26000C00086FFFCCF8091C00080648093C00006
:10F2700010E21093C6008091C00086FFFCCF809101
:10F28000C00080648093C0008BBEF3012791C45DF1
:10F29000DE4F2883CC52D140A22EBB24CC24DD24C7
:10F2A0000894611C711C811C911C8BBEF301879119
:10F2B000282E332444245524142D032DF22CEE241F
:10F2C000EA0CFB1C0C1D1D1D0894611C711C811C8B
:10F2D000911C8BBEF3013791C35DDE4F3883CD5255
:10F2E000D1400894611C711C811C911C8BBEF301E0
:10F2F0004791C25DDE4F4883CE52D1402DEF3FEFA4
:10F300004FEF5FEF620E731E841E951E0F947EF307
:10F3100030E23093C6008091C00086FFFCCF809120
:10F32000C00080648093C000C45DDE4F8881CC52F1
:10F33000D1400F947EF340E24093C6008091C0001C
:10F3400086FFFCCF8091C00080648093C000C25DC6
:10F35000DE4F8881CE52D1400F947EF350E250931D
:10F36000C6008091C00086FFFCCF8091C000806401
:10F370008093C000C35DDE4F8881CD52D1400F9491
:10F380007EF380E28093C6008091C00086FFFCCFB0
:10F390008091C00080648093C0009FEFE9169FEFCA
:10F3A000F90690E0090790E0190731F48EE092EE3B
:10F3B00060E00F942FF3DFC0D801C7018070907C0C
:10F3C000A070B0708050904CA040B040D1F52FEFAD
:10F3D0003FE340E050E0E222F32204231523C85D1E
:10F3E000DE4FA880B980CA80DB80C852D140AE0C05
:10F3F000BF1CC01ED11EAA0CBB1CCC1CDD1C88E18E
:10F4000092EE60E00F942FF3BB27A12F902F8F2D4A
:10F410000F947EF38E2D0F947EF330E23093C6006E
:10F420008091C00086FFFCCF8091C00080648093F3
:10F43000C0004EE34093C6008091C00086FFFCCF21
:10F4400087C08EE09EEFA0E0B0E0E822F9220A2318
:10F450001B239CE0E91694E9F90690E0090790E087
:10F46000190709F088C0C25DDE4FA881CE52D14095
:10F47000EA2EFF2400E010E0102F0F2DFE2CEE24CA
:10F48000C35DDE4FB881CD52D140EB0EF11C011DA2
:10F49000111DD601C50181709070A070B070DC01A3
:10F4A00099278827E80EF91E0A1F1B1F20EF30E05E
:10F4B00040E050E0A222B322C422D522F1E1AA0CFE
:10F4C000BB1CCC1CDD1CFA95D1F7EA0CFB1C0C1DF7
:10F4D0001D1D81E090E0A0E0B0E0282239224A2200
:10F4E0005B22E5E1220C331C441C551CEA95D1F744
:10F4F000E20CF31C041D151D57016801AA0CBB1C6E
:10F50000CC1CDD1C8FE192EE60E00F942FF3C8015C
:10F51000AA27BB270F947EF3BB27A12F902F8F2DF7
:10F520000F947EF38E2D0F947EF390E29093C6009D
:10F530008091C00086FFFCCF8091C00080648093E2
:10F54000C000AEE3A093C6008091C00086FFFCCF50
:10F550008091C00080648093C000C601AA27BB27A9
:10F560000F947EF3BB27AD2D9C2D8B2D0F947EF336
:10F570008A2D0F947EF3B0E2B093C6008091C00054
:10F5800086FFFCCF8091C00080648093C000CC5D7A
:10F59000DE4FE881F981C452D140CF01AA2797FDFF
:10F5A000A095BA2FABBFFC018791969160E00F94B4
:10F5B0002FF30F944DF3CC5DDE4F08811981C452B7
:10F5C000D1400E5F1F4FCC5DDE4F19830883C452BC
:10F5D000D140CA5DDE4F28813981C652D1402933DE
:10F5E000310509F417CB84E090E0A0E0B0E0680EAC
:10F5F000791E8A1E9B1EC9CD80E393EE62E00F94B4
:10F6000066F384E292EE60E00F942FF38091C000E5
:10F6100087FFFCCF1091C6001F751093C600809124
:10F62000C00086FFFCCF8091C00080648093C00042
:10F630000F944DF3812F81548A3108F036C116346E
:10F6400009F495C0173490F4133409F44EC01434FF
:10F6500030F41134F1F0123409F01DC130C014340B
:10F6600009F459C0153409F016C16BC01A3409F4F5
:10F67000C4C01B3438F4173409F48FC0183409F0AF
:10F680000AC1A1C01B3409F4D2C01C3409F003C163
:10F69000E8C08FEF81B90DC082B1809582B980E05A
:10F6A00090E0E0EDF7E03197F1F70196883C9105A5
:10F6B000C1F78091C00087FFEFCF12B8EFC08FEF86
:10F6C00084B90DC085B1809585B980E090E0E0ED0A
:10F6D000F7E03197F1F70196883C9105C1F78091E9
:10F6E000C00087FFEFCF15B8D9C08FEF87B90DC025
:10F6F00088B1809588B980E090E0E0EDF7E031973F
:10F70000F1F70196883C9105C1F78091C00087FF11
:10F71000EFCF18B8C3C08FEF8AB90DC08BB18095F9
:10F720008BB980E090E0E0EDF7E03197F1F70196DA
:10F73000883C9105C1F78091C00087FFEFCF1BB8CF
:10F74000ADC08FEF8DB90DC08EB180958EB980E0C0
:10F7500090E0E0EDF7E03197F1F70196883C9105F4
:10F76000C1F78091C00087FFEFCF1EB897C08FEF21
:10F7700080BB0DC081B3809581BB80E090E0E0ED5F
:10F78000F7E03197F1F70196883C9105C1F7809138
:10F79000C00087FFEFCF11BA81C08FEF83BB0DC0D0
:10F7A00084B3809584BB80E090E0E0EDF7E0319792
:10F7B000F1F70196883C9105C1F78091C00087FF61
:10F7C000EFCF14BA6BC08FEF809301010FC080910F
:10F7D000020180958093020180E090E0E0EDF7E087
:10F7E0003197F1F70196883C9105C1F78091C000EF
:10F7F00087FFEDCF1092020151C08FEF809304017B
:10F800000FC08091050180958093050180E090E014
:10F81000E0EDF7E03197F1F70196883C9105C1F7EB
:10F820008091C00087FFEDCF1092050137C08FEFA8
:10F83000809307010FC08091080180958093080193
:10F8400080E090E0E0EDF7E03197F1F70196883C39
:10F850009105C1F78091C00087FFEDCF109208019C
:10F860001DC08FEF80930A010FC080910B0180951E
:10F8700080930B0180E090E0E0EDF7E03197F1F745
:10F880000196883C9105C1F78091C00087FFEDCFBC
:10F8900010920B0103C08FE292EEB9C98091C000B3
:10F8A00087FFFCCF8091C600B5C982E492EEAFC954
:10F8B0008CE191EEACC9AA24BB24933061F1943061
:10F8C00028F4913089F0923008F508C09530B1F1F4
:10F8D000953040F1963009F053C04EC02B3109F0FD
:10F8E0001FC991E06BE11CC9213041F0C15DDE4FC1
:10F8F0009881CF52D140291709F0E5C26227C15D36
:10F90000DE4F2883CF52D14092E00AC9B22FA0E047
:10F91000622793E005C9822F90E0A82BB92B6227BC
:10F9200094E0FEC82E3009F0CEC2622795E0C05D9B
:10F93000DE4F19821882C053D140F2C8E1E0F0E0F6
:10F94000EC0FFD1FC05DDE4FE880F980C053D14051
:10F95000EE0DFF1D208387010F5F1F4FC05DDE4F3F
:10F9600019830883C053D14062270A171B0709F087
:10F97000D7C8D80196E0D4C8261709F0A4C203C09E
:10F98000973009F0CDC899249981933109F4F2C0D8
:10F990009431C8F4963009F4B8C0973050F49230DE
:10F9A00009F4E6C0933009F458C0913009F0EDC174
:10F9B0003EC0913109F462C0923108F0D9C0903153
:10F9C00009F0E3C1D5C0983109F472C0993150F4FF
:10F9D000953109F4CFC0953108F45AC1963109F038
:10F9E000D4C156C19A3109F457C09A3108F47CC089
:10F9F0009B3109F446C09D3109F0C7C18D81803328
:10FA000011F090E00AC08F81882311F49EE105C0B7
:10FA1000813011F091E001C098E91A821B828D813A
:10FA20008C831D829E831F8227E030E0B2C11A8240
:10FA300088E08B8381E48C8386E58D8382E58E83E9
:10FA400089E48F8383E5888780E589878FE58A87C6
:10FA500082E38B872BE030E09CC18A81813941F0C1
:10FA6000823941F0803911F48FE005C080E003C095
:10FA700082E001C08AE01A828B8344C09924939467
:10FA800077C08D81882311F48EE12CC0813011F074
:10FA900081E028C088E926C01A82E1E0F0E089E030
:10FAA0008093570084918B831C8224E030E071C1E5
:10FAB0008B81803589F48C81883039F4E2E0F0E084
:10FAC00089E08093570084910DC0E0E0F0E089E088
:10FAD00080935700849106C0E3E0F0E089E08093D2
:10FAE000570084911A82DFCF8D81836C99E0E1E029
:10FAF000F0E0082E90935700E89507B600FCFDCF84
:10FB00001A821B8223E030E044C18A8190E0A0E0A9
:10FB1000B0E0582F4427332722278B8190E0A0E0C4
:10FB2000B0E0DC0199278827282B392B4A2B5B2B47
:10FB30008D8190E0A0E0B0E0282B392B4A2B5B2B85
:10FB40008C8190E0A0E0B0E0BA2FA92F982F8827F1
:10FB5000282B392B4A2B5B2B220F331F441F551F99
:10FB6000C05EDE4F288339834A835B83C052D14015
:10FB70001A820DC13A81CD5CDE4F3883C353D14028
:10FB8000CE5CDE4F1882C253D1408B81082F10E02B
:10FB9000CE5CDE4F48815981C253D140042B152BD6
:10FBA000933149F0C05EDE4F488159816A817B8183
:10FBB000C052D14063C0C05EDE4F288139814A8186
:10FBC0005B81C052D1402070203080EC380783E048
:10FBD000480780E0580750F483E0F90140935B0048
:10FBE00080935700E89507B600FCFDCFC05EDE4F5E
:10FBF000488159816A817B81C052D140DE011B96C8
:10FC000031E08C9111962C9111971296CB5CDE4FBE
:10FC10002883C553D140CC5CDE4F1882C453D140F9
:10FC200090E0CC5CDE4FE881F981C453D1408E2B4B
:10FC30009F2B0C01FA0160935B0030935700E8950D
:10FC400011244E5F5F4F6F4F7F4F02501040C9F637
:10FC500085E0C05EDE4FE880F9800A811B81C052DA
:10FC6000D140F70100935B0080935700E89507B6F9
:10FC700000FCFDCF81E180935700E8951A82C05EB9
:10FC8000DE4F488359836A837B83C052D1407FC053
:10FC9000FA80C95CDE4FF882C753D140CA5CDE4FA0
:10FCA0001882C653D1408B81C82EDD24CA5CDE4F3A
:10FCB00008811981C653D140C02AD12A1A8289816C
:10FCC000BE016D5F7F4F843121F59601C05EDE4F2E
:10FCD000E880F9800A811B81C052D1400BBFF70137
:10FCE00087919691DB018C9311969C936E5F7F4F69
:10FCF000D801C7010296A11DB11DC05EDE4F8883E9
:10FD00009983AA83BB83C052D14022503040F1F680
:10FD100036C0C05EDE4F288139814A815B81C05286
:10FD2000D1400894C108D108760100E010E00894A1
:10FD3000C11CD11C0894E11CF11C011D111DE20E17
:10FD4000F31E041F151F21BDBB27A52F942F832F42
:10FD500082BD2F5F3F4F4F4F5F4FF89A80B5DB0159
:10FD60008D93BD012E153F054007510761F7C05E19
:10FD7000DE4F288339834A835B83C052D14096018A
:10FD80002D5F3F4FFB01108204C080EC8A8322E08C
:10FD900030E08BE18093C6008091C00086FFFCCFED
:10FDA0008091C00080648093C000C15DDE4FF88107
:10FDB000CF52D140F093C6008091C00086FFFCCFA7
:10FDC0008091C00080648093C000432F3093C600B0
:10FDD0008091C00086FFFCCF8091C000806480933A
:10FDE000C000922F2093C6008091C00086FFFCCFF8
:10FDF0008091C00080648093C0008EE08093C60034
:10FE00008091C00086FFFCCF8091C0008064809309
:10FE1000C00065E1C15DDE4FE880CF52D1406E2564
:10FE200069276427FE01319610C090819093C60027
:10FE30008091C00086FFFCCF31968091C000806425
:10FE40008093C0006927215030402115310569F7A2
:10FE50006093C6008091C00086FFFCCF8091C000F7
:10FE600080648093C00085B1805885B9992081F461
:10FE7000C15DDE4F0881CF52D1400F5FC15DDE4FC3
:10FE80000883CF52D14090E0A0E0B0E00D9490F50F
:10FE900027982F9880E090E020ED37E0F901319726
:10FEA000F1F7019684369105C9F700008091C000F2
:10FEB0008D7F8093C00081E180935700E895EE2705
:10FEC000FF270994FFCF90E00D9490F597FB092E42
:10FED00007260AD077FD04D02ED006D000201AF4D1
:10FEE000709561957F4F0895F6F7909581959F4F96
:10FEF0000895A1E21A2EAA1BBB1BFD010DC0AA1F6B
:10FF0000BB1FEE1FFF1FA217B307E407F50720F082
:10FF1000A21BB30BE40BF50B661F771F881F991FFD
:10FF20001A9469F760957095809590959B01AC0146
:10FF3000BD01CF010895AA1BBB1B51E107C0AA1F39
:10FF4000BB1FA617B70710F0A61BB70B881F991F7A
:10FF50005A95A9F780959095BC01CD010895F9991E
:10FF6000FECF92BD81BDF89A992780B50895262FBE
:10FF7000F999FECF1FBA92BD81BD20BD0FB6F8948E
:0EFF8000FA9AF99A0FBE01960895F894FFCFF1
:040000033000E000E9
:00000001FF
